:020000040000FA
:020000001928BD
:08000800F92908208600080018
:100010008207C034F934A434B03499349234823431
:10002000F83480349034E334FE34F734FF30860003
:10003000080003138312850107309F008316A03048
:100040008500803086000A308E0082308100831265
:100050005F308500FF308600FA30A900063081004D
:100060008B168B17AF01861F2F140A30A1000230A8
:10007000A2000130A3000030A4000430A000A701BA
:10008000A801AA01AC01AB01AD01B201B301162078
:1000900005148511AC1850282B1C542816205628FE
:1000A000AD1C5428851F4E2821080520D02116207C
:1000B00085150511AC1860282B1C602816206428B3
:1000C000AD185E2822080520D021162005158510C0
:1000D000AC186E282B1C6E281620702823080520CB
:1000E000D021162085140510AC187A282B1C7A28EC
:1000F00016207C2824080520D0212008031D47282D
:1001000016200514851AB9288B16A80803198A2801
:10011000A80BA2288316FF3086008312061C01213B
:10012000861C1A21061D3321861D4C21061E6521C1
:10013000061A7621861E8121061F932183168030A0
:10014000860083122F1CB3282D1DB32826080F39D3
:10015000A400260E0F39A30025080F39A200250E92
:100160000F39A100AD012C1CB828AC18B828D92033
:1001700047288B12AB012F1CD828851FD9202D159D
:10018000851FCE282D18CF28A40A2408093C03185F
:10019000CB28A30AA4012D14AD14CF282D1083164B
:1001A00006168312AA01061E652183160612831203
:1001B00047283308163C0319F128861BE128B20AA8
:1001C000E428320803190029B30A3308163C031D3A
:1001D0000029330832022E14031D2E103308B200FA
:1001E0000029B20B0029B301851AFC282E1CFA281D
:1001F000AC1400292C1000290B302E1C0C30A1004F
:1002000008002708031D06293330A700A70B19296A
:10021000AC012A181129A40A0A3024020318A401E7
:1002200017290130A402031817290930A4008230CD
:10023000A80008002708031D1F293330A700A70BBB
:100240003229AC012A182A29A30A0A3023020318EA
:10025000A30130290130A302031830290930A3007B
:100260008230A80008002708031D38293330A70072
:10027000A70B4B29AC012A184329A20A0A302202F3
:100280000318A20149290130A202031849290930A3
:10029000A2008230A80008002708031D512933302E
:1002A000A700A70B6429AC012A185C29A10A0A300F
:1002B00021020318A10162290130A1020318622959
:1002C0000930A1008230A80008002A1875292708E3
:1002D000031D6C293330A700A70B7529851A7229D5
:1002E0002A1475290513E921051708002A1C8029FD
:1002F0002708031D7D293330A700A70B80292A106A
:1003000008002708031D86293330A700A70B922970
:100310002A188D29AD212C149229AC01A101A2012A
:10032000A301A4010800AC1CAC292708031D9A29CD
:100330003330A700A70BAC290513E9210517AB0142
:100340002F1CAC29210E2204A500A101A201230E1D
:100350002404A600A301A4010800210E2204A50084
:10036000230E2404A6008B120512E9212508BE21C4
:100370002608BE210516E9218B160800B0000830BA
:10038000B100B00D0318C6290512C82905160000D2
:10039000E921B10BC12908002030D1294030D129F1
:1003A0006330B400B40BD22908000430B4003130FB
:1003B000B500DA29B50BD929B40BD72908000430C8
:1003C000B4006330B500E429B50BE329B40BE1298F
:1003D00008000830B4006330B500EE29B50BED29F4
:1003E000B40BEB290800F630B600D521B60BF52981
:1003F0000800F0000308F10083120B1D19280B11EF
:1004000006308100A90B152AFA30A900200803192B
:10041000122AA00B152AA101A201A301A4012B14E9
:100420008B12152A0130AB06A70171088300F00E6C
:04043000700E090041
:02400E00103F61
:1042000043006F0070007900720069006700680069
:1042100074002000280043002900200032003000F4
:104220003100300020006200790020004D002E0097
:10423000590061006D0061006D006F0074006F0037
:00000001FF
